:020000040800F2
:1000000000090020E1040008351B0008391B000826
:100010008D1B0008391B0008611B0008E304000861
:10002000E3040008E3040008E3040008B13D00080D
:10003000E3040008E3040008E30400084D4300085B
:10004000E3040008E3040008E3040008E3040008F4
:10005000E3040008E3040008314100085D410008A2
:1000600089410008B5410008E1410008E3040008A7
:10007000E3040008E3040008E3040008E3040008C4
:10008000E3040008E3040008E3040008A52C0008CA
:10009000112D0008652D0008B92D00080D4200083B
:1000A000E3040008E3040008E3040008E304000894
:1000B000E3040008E3040008E3040008E304000884
:1000C000E3040008E3040008E3040008E304000874
:1000D000E30400087531000889310008E3040008D2
:1000E00075420008E3040008E3040008E304000884
:1000F000E3040008E3040008E3040008E304000844
:10010000E3040008E3040008E3040008E304000833
:10011000E3040008E3040008E3040008E304000823
:10012000E3040008E3040008E3040008E304000813
:10013000E3040008E3040008E3040008E304000803
:10014000E3040008E3040008E3040008E3040008F3
:10015000E3040008E3040008E3040008E3040008E3
:10016000E3040008E3040008E3040008E3040008D3
:10017000E3040008E3040008E3040008E3040008C3
:10018000E3040008E3040008E3040008E3040008B3
:10019000E3040008E3040008E3040008E3040008A3
:1001A000D0400B1CD1409C46203AD34018435242C9
:1001B00063469340184370479140031C90409C460F
:1001C000203A9340194352426346D3401943704743
:1001D00053B94AB9002908BF00281CBF4FF0FF31AE
:1001E0004FF0FF3000F07AB9ADF1080C6DE904CEA4
:1001F00000F006F8DDF804E0DDE9022304B0704702
:100200002DE9F0478C460D460446089E002B51D13F
:100210008A4217466DD9B2FA82FEBEF1000F0BD0AA
:10022000CEF1200C01FA0EF520FA0CFC02FA0EF7C2
:100230004CEA050C00FA0EF44FEA174A250CBCFBF9
:10024000FAF81FFA87F90AFB18CC45EA0C4508FBB7
:1002500009F3AB420AD9ED1908F1FF3280F023818E
:10026000AB4240F22081A8F102083D44ED1AA4B24D
:10027000B5FBFAF00AFB105544EA054400FB09F906
:10028000A14509D9E41900F1FF3380F00A81A145A5
:1002900040F2078102383C44A4EB090440EA0840DC
:1002A0000021002E61D024FA0EF400233460736024
:1002B000BDE8F0878B4207D9002E54D0002186E894
:1002C00021000846BDE8F087B3FA83F1002940F029
:1002D0008E80AB4202D3824200F2FA80841A65EB30
:1002E00003050120AC46002E3FD086E81010BDE883
:1002F000F08712B90127B7FBF2F7B7FA87FEBEF114
:10030000000F34D1EB1B3A0C1FFA87FC0121B3FB21
:10031000F2F8250C02FB183345EA03450CFB08F301
:10032000AB4207D9ED1908F1FF3002D2AB4200F21F
:10033000D1808046ED1AA3B2B5FBF2F002FB105556
:1003400043EA05440CFB00FCA44507D9E41900F17D
:10035000FF3302D2A44500F2B8801846A4EB0C0487
:1003600040EA08409DE731463046BDE8F087CEF1CF
:10037000200405FA0EF307FA0EF720FA04F83A0CF7
:1003800025FA04F448EA0308B4FBF2F14FEA1845F1
:1003900002FB11441FFA87FC45EA044501FB0CF3FC
:1003A000AB4200FA0EF409D9ED1901F1FF3080F0EB
:1003B0008A80AB4240F2878002393D44EB1A1FFA33
:1003C00088F5B3FBF2F002FB103345EA034500FB6E
:1003D0000CF3AB4207D9ED1900F1FF386FD2AB42F5
:1003E0006DD902383D44EB1A40EA01418FE7C1F173
:1003F000200722FA07F88B4005FA01F448EA0303C4
:1004000020FA07FE4FEA134CFD404EEA040EB5FBFE
:10041000FCF94FEA1E440CFB19551FFA83F844EA15
:10042000054509FB08F4AC4202FA01F200FA01FAB0
:1004300008D9ED1809F1FF3043D2AC4241D9A9F1F6
:1004400002091D442D1B1FFA8EFEB5FBFCF00CFBB0
:1004500010554EEA054400FB08F8A04507D9E418FA
:1004600000F1FF3529D2A04527D902381C4440EAC3
:100470000940A4EB0804A0FB02894C45C6464D4642
:1004800015D312D056B1BAEB0E0364EB050404FA8F
:1004900007F7CB401F43CC40376074600021BDE8B4
:1004A000F0871846F8E69046E0E6C245EAD2B8EB97
:1004B000020E69EB03050138E4E72846D7E740461A
:1004C00091E78146BEE7014678E702383C4445E7BC
:1004D000084608E7A8F102083D442BE7704700BF33
:1004E00002E000F000F8FEE772B6394880F30888B1
:1004F000384880F3098838484EF60851CEF200019A
:10050000086040F20000CCF200004EF63471CEF2EA
:1005100000010860BFF34F8FBFF36F8F40F2000000
:10052000C0F2F0004EF68851CEF200010860BFF331
:100530004F8FBFF36F8F4FF00000E1EE100A4EF6C1
:100540003C71CEF200010860062080F31488BFF3EE
:100550006F8F03F06BFC03F013FD4FF055301F4914
:100560001B4A91423CBF41F8040BFAE71C49194A67
:1005700091423CBF41F8040BFAE71A491A4A1B4B57
:100580009A423EBF51F8040B42F8040BF8E70020F2
:100590001749184A91423CBF41F8040BFAE703F0AF
:1005A00049FC03F02FFD144C144DAC4203DA54F80F
:1005B000041B8847F9E700F03FF8114C114DAC429D
:1005C00003DA54F8041B8847F9E703F031BC000054
:1005D0000009002000110020000000080001002098
:1005E00000090020284B000800110020781100208D
:1005F00078110020C4270020A0010008A0010008F5
:10060000A0010008A00100082DE9F04F2DED108A8F
:10061000C1F80CD0C3689D46BDEC108ABDE8F08FD0
:10062000002383F311882846A047002003F0A4F993
:1006300003F04AF900DFFEE7334B6FF013022DE9B8
:10064000F0416FF0670100241A7003225A709C7009
:10065000DC701C715C719C71DC711C7259729A7235
:10066000DC7203F04FFB074603F09CFB0546B8BB6A
:10067000264B9F4236D001339F4236D0244B27F081
:10068000FF029A4235D1F8B200F074FDA84642F25A
:10069000107400F0A5FF00F073FD064668B374BB4C
:1006A000464635B11B4B9F4203D003F073FB002439
:1006B0002646002003F030FB174B1B6913F0400364
:1006C00020D00EB100F0CCF801F012FA00F0AAFF31
:1006D00001F052F9204600F00FF900F0C1F8F9E7F7
:1006E0008046D6E780460446D3E704464FF001082B
:1006F000CFE780464FF47A74CBE70446D1E74FF456
:100700007A74CEE71C46DFE778110020010007B0BD
:10071000000008B0263A09B00004004808B501F00E
:1007200017F9A0F120035842584108BD07B5054B01
:1007300002211B88ADF8043001A801F019F903B0BB
:100740005DF804FBC8440008064991F8243033B131
:1007500000230822086A81F8243001F03FB9012003
:10076000704700BF981100202DE9F84F234C94F8F2
:1007700024300546884617468BBB2E46DFF87C9012
:10078000002F38D094F824A0BAF1000F05D1202210
:10079000FF214846266201F0A1F9CAF10805BD42D1
:1007A00028BF3D465FFA85FBAD0041462A4604EB73
:1007B0008A0001F081F994F82430A7EB0B079B44E1
:1007C0005FFA8BFBBBF1080F2E44A844FFB284F8FC
:1007D00024B0D5D1FFF7B8FF0028D1D108E0266AB0
:1007E00006EB8306B042C9D0FFF7AEFF0028C4D1A4
:1007F0000020BDE8F88F0120BDE8F88F9811002097
:1008000010B5202383F311881148C3680BB103F09E
:1008100017F900230F4A0E48012103F0F7F80023CF
:1008200083F311880C4C236813B12368013B2360C8
:10083000636813B16368013B6360084B1B7833B98D
:10084000636823B9022001F02DF93223636010BDE3
:100850008411002001080008C8120020C0110020E7
:1008600010B51C4B1C4953F8042F013200D110BDA8
:100870008B42F8D1194C1A4B22689A4228D9194B4D
:100880009B6803F1006303F5D0439A4220D203F042
:1008900055FA03F067FA002001F088F8124B0220A5
:1008A000187001F0F7F8114BDA690022DA61D969A2
:1008B00099699A619B6972B60D4A0E4B13601B6869
:1008C0002268202181F311889D4683F30888104710
:1008D00010BD00BFFC6700081C6800080468000821
:1008E000FF67000878110020C011002000100240AE
:1008F00008ED00E0006800082DE9F04F99B0B34C16
:1009000001902022FF2110A8A66801F0E7F8B04A64
:100910001378A3469BB9AF480121C360117020230F
:1009200083F31188C3680BB103F08AF80023AA4A45
:10093000A848012103F06AF8002383F31188019B82
:1009400013B1A64B019A1A60A54AA449019F0292CD
:10095000002313704B6099461C461D4698460120A3
:1009600001F098F8002F00F012829C4B1B68002BBE
:1009700040F00D8219B0BDE8F08F0220FFF7CEFEE7
:10098000002840F0FB81019BB9F1000F08BF1F4612
:10099000944B1B88ADF82C3002210BA800F0E8FF27
:1009A000DDE74FF47A7000F0D3FF031E0393EADB18
:1009B0000220FFF7B3FE82460028E4D0039B581EB6
:1009C000042800F2DD81DFE800F0030E11141700A7
:1009D00018A8052340F8343D042100F0C9FF54460F
:1009E0004FF0000856E004217848F6E704217E48DD
:1009F000F3E704217D48F0E71C24204600F0D8FFEF
:100A000004340B9004210BA800F0B2FF2C2CF4D17D
:100A1000E5E7002DB7D0002CB5D00220FFF77EFE11
:100A20000546002800F0AF8101206D4C00F0BEFFAC
:100A30000220207001F02EF84FF000095FFA89FAC9
:100A4000504600F0D3FF074658B1504600F0DEFF95
:100A500009F101090028F1D12C46A9460027644B71
:100A600097E701230220237001F00CF83E46DBF8E3
:100A700008309E4206D2304600F09AFF0130EBD19A
:100A80000436F4E7029B00261E70544BA9465E60B4
:100A90002C46374601F02AF815B1002C18BF002764
:100AA000FFF744FE5BE7002D3FF46DAF002C3FF4F1
:100AB0006AAF029B0220187000F0ECFF322000F0B9
:100AC00047FFB0F1000AC0F25E811AF0030540F062
:100AD0005A81DBF8082006EB0A03934200F25381A7
:100AE000BAF5807F00F24F8155450DDA4FF47A70E8
:100AF00000F02EFF0490049B002BC0F244813D4A7D
:100B0000049BAB540135EFE7C820FFF707FE05460D
:100B1000002800F038811F2E11D8C6F1200454455A
:100B200028BF544610AB26F0030022463149184432
:100B300000F0C2FF2246FF212E4800F0CFFF4FEA0F
:100B4000AA0A5FFA8AF22B493046FFF70DFE0446E7
:100B5000002800F01A8106EB8A0605469AE7022073
:100B6000FFF7DCFD00283FF40EAFFFF7EDFD002896
:100B70003FF409AF4FF0000A5346DBF808209245D6
:100B80001CD2BAF11F0F12D8109A01320FD02AF0DE
:100B9000030218A90A4452F8202C0B92184604228A
:100BA0000BA901F00BF80AF1040A0346E5E75046E9
:100BB000039300F0FDFE039B0B90EFE718A80421C0
:100BC00040F84C3D00F0D4FE64E700BF78110020EF
:100BD000C41200208411002001080008C81200205F
:100BE000C0110020CA4400087C11002080110020A0
:100BF000CC440008C411002018A8002340F8343D5C
:100C0000642100F0ADFE00287FF4BDAE0220FFF7A6
:100C100085FD00283FF4B7AE0B9800F009FF18AB34
:100C200043F8480D04211846CCE718A8002340F8E3
:100C3000343D642100F094FE00287FF4A4AE02202D
:100C4000FFF76CFD00283FF49EAE0B9800F0F2FE1B
:100C500018AB43F8440DE5E70220FFF75FFD0028DD
:100C60003FF491AE00F0ECFE18AB43F8400DD9E72D
:100C70000220FFF753FD00283FF485AE0BA9142096
:100C800000F0E4FE824618A8042140F83CAD00F0D4
:100C90006FFE51460BA895E7322000F059FEB0F1E7
:100CA000000AFFF670AE1AF0030F7FF46CAEDBF8AB
:100CB00008200AEB080393423FF665AE0220FFF7D7
:100CC0002DFD00283FF45FAE2AF0030AC244D04550
:100CD0003FF4E0AE404600F06BFE04210A900AA803
:100CE00000F046FE08F10408F1E74FF47A70FFF7D0
:100CF00015FD00283FF447AEFFF726FD00283FF41E
:100D0000AEAE109B01330CD0082210A90020FFF7D3
:100D10002BFD00283FF4A3AE2022FF2110A800F0F5
:100D2000DDFEFFF703FD642002F02CFE22E6002D1D
:100D30003FF429AE002C3FF426AE18A8002340F85B
:100D4000343D642100F00CFE824600287FF41BAE87
:100D50000220FFF7E3FC00283FF415AE0390FFF7F5
:100D6000E5FC052002F00EFE0B9800F0C9FE00F035
:100D7000BDFE039B57461C461D46F0E5054689E629
:100D80004FF00008FFE52546FDE52C4667E600200C
:100D900000F0DEFD0490049B002B01DA00F098FCCB
:100DA000049B002BFFF6DEAD012000F06BFE049BE0
:100DB000213B122B3FF6D3AD01A252F823F000BF26
:100DC0007B090008A3090008130A00085F0900084E
:100DD0005F0900085F090008A70A0008990C0008CD
:100DE0005F0B0008F90B00082B0C0008590C0008D9
:100DF0005F090008710C00085F090008EB0C00088F
:100E0000950A00085F0900082F0D000809490B68C2
:100E100049F269009AB21B0C00FB0233064A0B60D0
:100E2000136844F2506198B21B0C01FB0030106053
:100E300080B27047101100200C11002010B5002165
:100E40001022044600F04AFE034B03CB2060616091
:100E50001868A06010BD00BFACF7FF1FF0B51F4CB5
:100E6000BBB000F0A7FEA368C31AF92B30D906ADBA
:100E70002346A06028220021284601F029FC04F125
:100E80000E0000F023FE0023C6B2591D5F1CDBB22A
:100E9000B3424FEAC10107DA0E3323440822284641
:100EA00001F016FC3B46F0E7012303930823207B67
:100EB00002930B4B0193C1F3CF01302305910093B3
:100EC0000146049503A3D3E90023064801F0D0F9B5
:100ED0003BB0F0BD78F6339F93CACD8D1023002030
:100EE0001D230020E822002070B50D4614461E4642
:100EF00001F064F950B9022E0ED1012C0CD112A3CD
:100F0000D3E90023C5E90023012070BD052C14D0CE
:100F100003D8012C09D0002070BD282C09D0302C1A
:100F2000F9D10BA3D3E90023ECE70BA3D3E900230A
:100F3000E8E70BA3D3E90023E4E70BA3D3E90023FD
:100F4000E0E700BFAFF30080401DA12026812A0BFF
:100F500078F6339F93CACD8D9E6AC421818A46EE6E
:100F600026417272DF25D7B7F017304A39059E56F1
:100F700038B504460D46034620222846002101F0DC
:100F8000A7FB22792346032A28BF032203F8042F54
:100F900028460222202101F09BFB62792346072A82
:100FA00028BF072203F8052F28460322222101F03B
:100FB0008FFBA2792346072A28BF072203F8062FB2
:100FC00028460322252101F083FB284604F108036B
:100FD0001022282101F07CFB382038BD2DE9F04F8C
:100FE000ADF5017D21AE0EAD40F2791280460F467F
:100FF0003046002100F072FD48220021284600F012
:101000006DFD00F0D7FD594B4FF47A72B0FBF2F052
:10101000186093E80700012385E807002B740DF1A1
:101020005A0000236B74FFF709FF032385F8203073
:10103000EC2385F8213007AB18464D4903F0F0F951
:101040001B2228643146284685F83C20FFF790FF94
:1010500012AB044601460822304601F039FB082253
:10106000A1180DF14903304601F032FB0DF14A039E
:10107000082204F11001304601F02AFB13AB2022B4
:1010800004F11801304601F023FB14AB402204F1B7
:101090003801304601F01CFB16AB082204F1780140
:1010A000304601F015FB0DF15903082204F18001CF
:1010B000304601F00DFB04F1880A0DF15A0904F5E0
:1010C000847B4B465146082230460AF1080A01F05B
:1010D000FFFAD34509F10109F3D11BAB08225946A8
:1010E000304601F0F5FA04F588744FF0000995F8E0
:1010F00034304B4510D84FF0000995F83C304B4543
:1011000015D92B6C21464B440822304601F0E0FAF9
:10111000083409F10109F0E7AB6B21464B44082282
:10112000304601F0D5FA083409F10109DFE7E31D83
:10113000C3F3CF03F97E0593002304960393BB7E8C
:101140000293193701230093019706A3D3E90023E3
:10115000404601F08DF80DF5017DBDE8F08F00BF30
:10116000AFF300809E6AC421818A46EED01200202F
:10117000E0450008014B1870704700BFDC120020EA
:10118000F0B52E4B1C7B85B02CB12D4B0E221A8155
:10119000002005B0F0BD2B4A1068516802AB03C3B4
:1011A00008230DEB03022849284803F01BF90546E4
:1011B00030B9234B26480A221A8100F0B3FCE7E736
:1011C0000369B3F5663F07D91D4A22480B211181F7
:1011D000194600F0A7FCDBE7418BB1F57B7F08D017
:1011E000174B1D480C221A814FF47B7200F09AFCB9
:1011F000CEE71A4A15490244103B20469E1A00F0D9
:10120000DDFC3246074605F11801204600F0D6FC09
:10121000AB689F4202D1EB6898420AD0084B0D227E
:101220001A8100903B46EA68A9680D4800F07AFCF4
:10123000AEE70C4800F076FC0120AAE7102300205E
:10124000D0120020D0440008DC970300006800089A
:10125000D8440008E4440008F64400080898FFF762
:10126000144500083D4500082DE9F04FAFB006AF2A
:1012700080460D4600F0A2FF044600286CD12B7E6C
:10128000022B18D1EB8A012B15D100F093FC81467B
:10129000FFF7BCFD4FF4C873BF4EB0FBF3F209F586
:1012A000167902FB1300EB7E19FA80F0306093B9D7
:1012B000BA4B00221A70A437BD46BDE8F08F07F183
:1012C0000C031C440094002308224FEAC90128465D
:1012D00001F062F84C46AB8A013BA3425FFA84F905
:1012E0000BD904F10109B9F1110FE8D1AC4BAD4AAA
:1012F00040F23911AC4803F047F807F11C00FFF742
:101300009DFD224607F11C0107F10C0003F05AF87D
:1013100003460028CCD1B9F1100F07D09F4B83F8BA
:1013200000903368A3F516733360C4E707F1A00299
:10133000014602F8950D28460092072201F02CF88C
:10134000F97A7F2904DD994B964A4FF4A871D1E7C9
:10135000404600F017FFAEE7EB8A052B00F02E8128
:1013600006D8012BA7D129464046FFF737FEA2E752
:10137000282B3DD0302B9ED16B7E8D4C0133627B70
:10138000DBB29342EA4640F00081EA7E237B9A4238
:1013900040F0FB8007F1A003002623F8846D1022A3
:1013A000009331460123284600F0F6FFB5F814807B
:1013B000A8F102081FFA88F808F1030323F00303D9
:1013C0000A3323F00703ADEB030D0DF11809334683
:1013D0009BB2B11C98454FEAC10106F101066DDDD3
:1013E0004B44009308220023284600F0D5FFEEE787
:1013F000AB8A013B9BB2C92B3FF65DAF6C4E347B91
:101400004CBB06F10C0300930822234621462846D4
:1014100000F0C2FFAB8A04F10109013BE4B29C4237
:101420004FEAC90109DA0E3434440094002308223B
:10143000284600F0B1FF4C46ECE700230022C6E945
:1014400000230023B36086F8D730C6F8D830337B4A
:101450000BB9EB7E3373002407F11C0607F10C0374
:10146000082221463046FC603C617C6101F030F985
:101470003B7C04F10109A3424FEAC90107D97B690A
:1014800008222344304601F023F94C46F0E7C1F32B
:10149000CF010023E87E059104960393AB7E02936F
:1014A0001935282301460093019539A3D3E9002378
:1014B000404600F0DDFEFFF7D1FCFCE694F8D700D3
:1014C00000F094FAD4F8D83006461BB994F8D70047
:1014D00000F09CFAD4F8D83043449E4204D294F8E9
:1014E000D700013000F092FA324B4FEA980B0025FA
:1014F000AAB25A45104616DA5AB994F8D72042B91A
:10150000D4E900120A4304D1D9F800201A60013549
:10151000EEE7226859F820107B6002EB800000F0B3
:101520004DFA7B68F3E7D4E90023D4F8D85012EBE6
:10153000080043F10001C4E90001454494F8D700D4
:10154000C4F8D85000F052FA854209D394F8D73045
:10155000013384F8D730D4F8D8309E1BC4F8D86053
:10156000B8F1FF0F0ADC134B00201968207300F05C
:1015700025FAFFF705FE08B1FFF772F923680E4A56
:101580009B0A013313810023A360D54693E600BF75
:1015900026417272DF25D7B7E4220020E122002025
:1015A0004C450008FC450008A5450008C745000853
:1015B0001023002000110020D0120020BFF34F8F15
:1015C0000549064BCA6802F4E0621343CB60BFF3DF
:1015D0004F8F00BFFDE700BF00ED00E00400FA05FB
:1015E00008B54FF000530B4A196891420AD10A4AD4
:1015F000597D117009481B7D0373C92208490E30BB
:1016000000F05AFAE02200214FF00050BDE80840F7
:1016100000F064BA9AAD44C5DC120020102300200B
:101620001600002030B5204C2049214885B0022307
:10163000637104230025ADF808300123ADF80C5088
:1016400007228DF80C308DF80B301A4B4B608DF85B
:101650000A2001F07BFE184B019500931749184BA7
:1016600018484FF4805200F057FD174B1978254663
:1016700011B1144800F086FD00F09CFA0446FFF713
:10168000C5FB4FF4C87304F51674B0FBF3F202FB0C
:1016900013000E4B14FA80F0186002F083FB08B1BF
:1016A0000F232B8105B030BDD01200200411002083
:1016B0001824002003000600E90E0008E0120020B4
:1016C00069120008E8220020DC120020E422002039
:1016D0002DE9F04F94A7D7E900670FF25429D9E913
:1016E00000898D4C93B0DFF850B2DFF850A220464D
:1016F00000F00AFE0CAD079098B310220021284696
:1017000000F0ECF9079B197B4FF0000261F3030234
:1017100019468DF8302051F8040F49680EAA03C20B
:101720001B680D9A63F31C029DF830300D9243F054
:1017300020038DF8303000232A461946584601F020
:1017400015FE079030B9204600F0E2FD079B8AF8AD
:101750000030CCE79AF80030072B3EDC01338AF8E2
:10176000003018220021284600F0B8F9DFF8C8A19F
:10177000002319462A46504601F020FE014680BB50
:10178000102208A800F0AAF94FF09042536983F0A4
:101790001003536100F010FA0B4612A9024611E93A
:1017A00003000DF1240E8EE803009DF83410C1F300
:1017B000030089064CBF0E99BDF838108DF82C0037
:1017C00046BFC1F31C0141F00041C1F30A01089179
:1017D000204608A900F0E2FFCAE7204600F098FD85
:1017E000BFE7204600F0EAFC824600284AD1DFF835
:1017F00050B100F0DFF9DBF80030984242D300F03E
:10180000D9F90790FFF702FB079A8DF820A04FF453
:10181000C87302F51672B0FBF3F101FB130012FA64
:1018200080F0CBF80000DFF81CB19BF8001011B974
:1018300001238DF8203028460791FFF7FFFA07991A
:10184000C1F1100A5FFA8AFABAF1060F28BF4FF009
:10185000060A524629440DF1210000F02DF90AF143
:101860000103049308AB0393182302932B4B0193BA
:101870000123009332463B46204600F0A1FC0023A2
:101880008BF8003000F096F9254ADFF8BCA0136809
:10189000C31AB3F57A7F32D3106000F08DF9024697
:1018A0000B46204600F03AFD204600F087FC30B39E
:1018B0009AF80C30DFF894B0002B14BF03230223F6
:1018C0008BF8053000F076F94FF47A732946B0FBB7
:1018D000F3F0CBF800005846FFF74AFB1823073017
:1018E0000293104B0193C0F3CF0040F255130490C4
:1018F0000093039542464B46204600F061FC9AF85F
:101900000C300BB1FFF7AAFA9AF80C30002B7FF4D9
:10191000EAAE13B0BDE8F08FE8220020E0220020FC
:10192000F0230020F4230020401DA12026812A0B53
:10193000F1C6A7C1D068080F18240020F5230020A5
:10194000E4220020E122002010230020D0120020F9
:1019500008B5012002F016F84FF0FF3008BD000076
:1019600008B5012002F00EF84FF0FF3008BD00006E
:1019700000231B68FFDE000070B502F0B9F8094CC7
:10198000094E2070002530682378834208D902F080
:10199000ABF8336805440133B5F5D04F3360F2D36B
:1019A00070BD00BF14240020F823002002F02EB9DF
:1019B00000F1006000F5D0400068704707B502AB49
:1019C00000F1006043F8041D0422194600F5D040E0
:1019D00002F0C8F803B05DF804FB000000F10060FD
:1019E000920000F5D04002F0BDB80000054B1A6827
:1019F000054B1B789B1A834202D9104402F074B83D
:101A000000207047F82300201424002038B5074D2B
:101A100004462868204402F06DF828B9286820445C
:101A2000BDE8384002F078B838BD00BFF823002088
:101A30000020704700F10050A0F654000068704785
:101A4000014B1868704700BF002004E030B5013832
:101A50000B4D0A180B46934210D215F9014F581C32
:101A60001CB1034600F8014CF5E72C2482421C709F
:101A700002D93F22981C5A70401A30BD1846FBE725
:101A80003F460008022802BF4FF0904310229A619F
:101A900070470000022802BF4FF090434FF48012BD
:101AA0009A617047022801BF4FF09042536983F05A
:101AB000100353617047000010B50023934203D018
:101AC000CC5CC4540133F9E710BD00000246034664
:101AD000981A13F9011B0029FAD1704702440346F2
:101AE000934202D003F8011BFAE7704770470000E9
:101AF000024B4FF461421A60704700BFFC23002084
:101B0000074B10B50021044618221846FFF7E6FFE0
:101B100004600146BDE81040002001F015BE00BF82
:101B2000FC2300200FB4002004B070470EB4002046
:101B300003B07047FEE7000000B59BB0EFF30981EA
:101B400068226846FFF7B8FFEFF30583034B9A6BF3
:101B50009A6A9A6A9A6A9A6A9B6AFEE700ED00E0BE
:101B600000B59BB0EFF3098168226846FFF7A4FF38
:101B7000EFF30583044B9A6B9A6A9A6A9A6A9A6A97
:101B80009A6A9B6AFEE700BF00ED00E000B59BB0DB
:101B9000EFF3098168226846FFF78EFFEFF30583B4
:101BA000034B5A6B9A6A9A6A9A6A9A6A9B6AFEE728
:101BB00000ED00E002F062B802F03CB830B5084D2C
:101BC0000A4491420BD011F8013B09245840013CD2
:101BD000F7D040F300032B4083EA5000F7E730BD15
:101BE0002083B8ED0246006848B103681360D388CB
:101BF000118901339BB29942D38038BF138170475A
:101C000070B588B00D460446202200216846FFF7D3
:101C100065FF20460495FFF7E5FF054658B16B4682
:101C2000044608AE1A4603CAB242206061601346F9
:101C300004F10804F6D1284608B070BD2DE9F04142
:101C400030B9274B274A40F2C531274802F09CFBA8
:101C50000B7C23B9254B234A40F2C631F5E7C66910
:101C600086B9C161BDE8F081002B29DA930CAB4243
:101C700029D1B44201D10C60F3E7C8F800100C6020
:101C8000BDE8F0814B6823F06047BD0C4FEAD37E7E
:101C9000C3F3807C15EA230538BF3D46B046344681
:101CA0006368BEEBD37F23F06042DDD1974203D15E
:101CB000C3F380739C450AD1974205E01C46EFE7C9
:101CC000AA4206D013469D422CBF00230123002BBD
:101CD000CFD12368A046002BF0D12160BDE8F08170
:101CE000DC480008D046000894490008B5490008BF
:101CF00008B5034A034B044840F25E3102F044FB4E
:101D0000AC460008544900089449000808B5036827
:101D10000B60C388016033B9044B054A05484FF492
:101D2000C76102F031FB013BC38008BD24490008B4
:101D3000204700089449000870B50C4600F10C05D6
:101D4000616831B9E38A61F30903E382002000216D
:101D500070BD0E682846FFF7D9FF6660F0E7000007
:101D600008B5426832B10B4B0B4A0C4840F22F4188
:101D700002F00AFBC37DC3F38401013161F38603E2
:101D8000C375C38A62F30903C3821B0A62F3C713D4
:101D9000C37508BD70490008DC4600089449000876
:101DA0002DE9F047089E32B91F4B204A204840F2E7
:101DB000395102F0E9FA01F007054FEAD6082A4442
:101DC00006F0070600EBD1004FF47F49954201D1A0
:101DD000BDE8F08705F0070E06F0070AD6457746FE
:101DE00038BF5746C7F10807511BEC088F4228BF80
:101DF0000F46045D08EBD60104FA0EF413F801C097
:101E000029FA07FE24FA0AF45FFA8EFE8CEA04042B
:101E10004EFA0AFE04EA0E048CEA040C03F801C030
:101E20003D443E44D2E700BFF0480008F4460008B5
:101E3000944900082DE9F04106460F4600254FF66B
:101E4000FF7441F221082A4630463946FEF7A8F9C8
:101E5000C0B284EA0024082314F4004F4FEA44047B
:101E6000A4B203F1FF3318BF84EA080413F0FF03A0
:101E7000F2D10835402DE6D12046BDE8F0810000C2
:101E800010B50A4441F22104914200D110BD11F86D
:101E9000013B80EA0320082310F4004F4FEA400082
:101EA00080B203F1FF3318BF604013F0FF03F3D19A
:101EB000EAE700002DE9F04F85B08A468DE80C0076
:101EC000BDF83C40814630B9494B4A4A40F26E3138
:101ED000494802F059FA11F0604F04D0474B454A87
:101EE00040F26F31F4E7009B002B7ED024B10E9BB3
:101EF000002B7AD0072C28D809F10C00FFF772FECE
:101F0000054628B96FF00205284605B0BDE8F08FF8
:101F100014220021FFF7E2FD22460E9905F1080088
:101F2000FFF7CAFD631C2B74009B1B782C4403F045
:101F30001F0363F03F0323724AF000436B6029469E
:101F40004846FFF77BFE0125DEE7019B1B0A4FF0A9
:101F50000008029300F10C034FF0800B4646454603
:101F600003930398FFF73EFE07460028CAD01422C9
:101F70000021FFF7B3FDB6BB9DF804303B729DF81E
:101F800008307B7202220E9B711E1944B4420AD99A
:101F9000B8180132D2B211F801EF80F808E001362A
:101FA000072AB6B2F2D1009B197801F01F01B442A2
:101FB00008BF4FF0400BB81841EA48114BEA010343
:101FC000037201324AF000437B603A743946484656
:101FD000FFF734FE0135B4422DB288F001084FF00E
:101FE000000BBED190E70022CDE76FF001058BE733
:101FF000DC480008C0460008944900080049000871
:102000002DE9F0471E46CB8A9146C3F30902062A02
:1020100080460F4619D013460021B0B28DB25A192E
:1020200092B2052A09D9A84210D8FA8A034463F368
:102030000902FA820120BDE8F087A842F3D93A44A8
:1020400019F8014094760131E8E70025FB8A7C68A5
:10205000C3F30900821F1C23B2FBF3FA03FB1A2A05
:102060001FFA8AF27CB301212368002B39D1B31FF8
:1020700003441C20B3FBF0F301339BB299420CD212
:10208000BAF1000F09D14046FFF7ACFD08B1C0F826
:1020900000A0206008B304460022B6B24FF0000A48
:1020A000B54230D2691E49441346E01801339BB251
:1020B00011F801EF80F804E001351C2BADB214D00B
:1020C000AE42F2D8ECE74046FFF78CFD044608B17B
:1020D000002303607C60002CDED16FF00200BDE8BD
:1020E000F087013189B21C46BEE7AE42D8D94046DE
:1020F000FFF778FD08B1C0F800A020600028ECD000
:1021000004460022CCE7FB8AC3F30902164466F3B7
:102110000903FB828EE70000F8B50E4615461F4600
:10212000044628B9144B154A15484F2102F02CF9E2
:1021300024220021FFF7D2FC069B6360079B2362E9
:102140006A094FF6FF739A424FF0000028BF1A4603
:10215000A7602070A061E06197B204F10C05824293
:1021600005D100232B6027826382A382F8BD2E60F5
:10217000013035462036F2E7D84800084C460008C2
:102180009449000808B528B9084B094A7321094841
:1021900002F0FAF8037823B94BB2002B01DD01708D
:1021A00008BD054B024A7D21F1E700BFDC4800086D
:1021B00058460008944900082048000800787047F5
:1021C0002DE9F7430D9EBDF828900B9D9DF83040FA
:1021D000BDF8388007461946104616B9B8F1000F09
:1021E00043D11F2C41D83B78D3B9B8F1070F39D868
:1021F00039F0030339D1424631464FF6FF70FFF7FD
:102200003FFE4FEA092920F0010009F4407940041B
:1022100049EA0464400C44EA40244FF6FF730DE0A1
:1022200043EA0923B8F1070F43EA0464F5D9FFF73D
:1022300001FE42463146FFF723FE03468DE840018A
:102240002A4621463846FFF735FE0DB9FFF750FD07
:102250002B780133DBB21F2B88BF00232B7003B018
:10226000BDE8F0836FF00300F9E76FF00100F6E7D7
:102270002DE9F7430E9F0B9D9DF83480BDF83C601F
:1022800081469DF8300007B9C6BB1F2836D899F89B
:1022900000E0BEF1000F34D00C0244F080049DF841
:1022A000281044EAC83444EA014444EA0E04072EE4
:1022B00044EA006415D919461046FFF7BBFD3246C3
:1022C0003946FFF7DDFD0346019600972A46214671
:1022D0004846FFF7EFFDB8F1010F0CD125B9FFF724
:1022E00007FD4FF6FF73EFE72B780133DBB21F2BAF
:1022F00088BF00232B7003B0BDE8F0836FF00100AE
:10230000F9E76FF00300F6E7C06900B104307047E9
:10231000C1690B68C3610C30FFF7F8BC2DE9F84FB9
:10232000D0F818A0DFF86C80054616461F465446C4
:102330004FF0000900F10C0B0CB9BDE8F88FD4E99F
:102340000223B21A67EB0303994508BF90451FD2D9
:10235000AB699C42214628460DD1FFF7EDFCAB69E5
:102360001B68AB6121465846FFF7D0FCAC69234699
:10237000A2461C46E0E7FFF7DFFC2368CAF80030FE
:1023800021465846FFF7C2FC5446DAF80030EFE722
:102390002368EDE780841E002DE9F04F8BB00D46D9
:1023A00014460793DDF850908246002800F06481BF
:1023B000B9F1000F00F06081531E3F2B00F25C81E9
:1023C000012A03D1079B002B40F05681BAF8146014
:1023D000F6000023B5420893099380F053812B192E
:1023E0009E420AD2761B16F0FF0607D1AB4BAC4AD1
:1023F00040F26751AB4801F0C7FF2646DAF80C30CF
:1024000023B9DAF81030002B00F0A5802F2D31D839
:10241000C5F1300846454FF000032CBF5FFA88F83D
:10242000B0460093294608AB4246DAF80800FFF7A9
:10243000B7FCA6EB08074544FFB2BAF8143003F125
:102440000053063BDB000293DAF80C3005934FF0A3
:10245000300B059B002B51D087B9DAF8100000280B
:1024600061D0002F5FD0AB4550D98F4B8C4A40F2E2
:10247000A651BFE737464FF00008DEE7029B23B9BD
:102480008A4B874A4FF4B161B4E7029BE02B28BF27
:10249000E02306935B44AB4204931DD95B1B9F4230
:1024A00026BFDBB203930397AB4504D97E4B7C4A2E
:1024B00040F291519EE70598CDF8008008ABA5EB5E
:1024C0000B01039A0430FFF76BFC039B9844FF1A3F
:1024D0001D445FFA88F8FFB2049B9B4504D3744BFC
:1024E0006F4A40F29B5185E7029B069ADDF810B0D7
:1024F0009B1A0293059B1B680593AAE7029BBB42AC
:10250000ABD26C4B664A40F2A15173E7CDF8008024
:102510003A46A5EB0B0108ABFFF742FCB8443D443B
:102520005FFA88F80027BAF81430B5EBC30F04D966
:10253000614B5B4A40F2B1515CE7B8F1400F04D9FE
:102540005E4B574A40F2B25154E767B15C4B544A74
:1025500040F2B3514EE70093324608AB2946DAF811
:102560000800FFF71DFC731E3F2B35B201D8A642B1
:1025700004DD544B544A40F235213BE760070AD052
:102580000AAB03EBD401624211F8083C02F00702E7
:10259000134101F8083C082C21D9102C21D9202CFA
:1025A0008CBF08230423079A002A6DD0B4EBC30F15
:1025B0006CD0082C04F1FF3215D89DF8203023FA96
:1025C00002F2D10706D54FF0FF3202FA04F423439A
:1025D0008DF820309DF8203089F800304EE001233E
:1025E000E1E70223DFE7102C11D8BDF8203023FAF1
:1025F00002F2D20706D54FF0FF3202FA04F4234369
:10260000ADF82030BDF82030A9F8003036E0202C9D
:102610000ED8089921FA02F2D30705D54FF0FF33FF
:1026200003FA04F40C430894089BC9F8003025E031
:10263000402C1CD0DDE9086730463946FDF7B0FD77
:10264000002100F0010050EA01030BD022460120D6
:102650000021FDF7B1FD404261EB410106430F430C
:10266000CDE90867DDE90823C9E9002306E0174B37
:10267000154A4FF42071BDE66FF0010528460BB0F6
:10268000BDE8F08F1D46F9E7012CA3D0082CA1D995
:10269000102CB7D9202CE5D8C6E700BF2C4700087E
:1026A00004470008944900084E4700083B470008CB
:1026B000734700089B470008C2470008F04700081E
:1026C00008480008224800088446000820480008FE
:1026D00030B585B030B9244B244A40F2B1212448AA
:1026E00001F052FE23B9234B204A40F2B221F6E713
:1026F000402A04D9204B1D4A40F2B621EFE722B907
:102700001D4B1A4A4FF42F71E9E70024012A029465
:10271000039417D11B788DF8083053070AD004AB07
:1027200003EBD203554213F8084C05F00705AC4003
:1027300003F8084C00910346002102A8FFF730FB84
:1027400005B030BD082AE5D9102A03D81B88ADF89A
:102750000830E2E7202A02D81B680293DDE7D3E9BC
:102760000045CDE90245D8E75C48000898460008D6
:1027700094490008774800082048000870B50C46C6
:1027800000F10C05E16819B9A1602161A18270BD59
:102790000E682846FFF7BAFAE660F3E72DE9F04F36
:1027A000D1F8009091B0C9F3C01604460D46CDE9AA
:1027B0000223002E50D0C9F3C03BC9F30626B9F15D
:1027C000000F80F29F8119F0C04F40F09B812B7B5E
:1027D000002B00F09781BBF1020F03D02278B242A8
:1027E00040F0938109F07F02BBF1020F059236D1D0
:1027F00019F07F0FC9F30F2A01D10AF0030A2B4405
:102800007606059A93F8038046EA0B4646EA824626
:102810005FEAD81346EA0A06069300F09A8000227F
:10282000002310A961E90823059B009367685B46B4
:1028300052462046B847002800F08880A7698FB923
:10284000314604F10C00FFF7DBF90746D0B96FF011
:10285000020011B0BDE8F08F4FF0020BAFE7C9F3F3
:10286000074ACCE73B699E420DD03F68002FF9D163
:10287000314604F10C00FFF7C3F907460028E6D003
:10288000A3693B60A761DDE90801FFF7D3FAB882CD
:10289000F97D08F01F06C1F38401711A89B20FFA9D
:1028A00081FED7E90223BEF1000FB8BF01F1200E6F
:1028B000C9F30461B8BF0FFA8EFE079152EA030113
:1028C00000F02F81DDE90201801A61EB030102466D
:1028D0000B469F480021994208BF9042C0F02181D9
:1028E000069B002B3FD0BEF1010F00F31A8118F0B8
:1028F000400F38D0DDE90223C7E90223202200215E
:102900000DEB0200FFF7EAF8DDE90223CDE9082329
:102910002B1D0A932B7BADF836A0013BDBB2ADF843
:1029200034309DF81C308DF83A309DF814308DF815
:102930003B3020468DF838B08DF83960A36808A97F
:1029400098473846FFF70CFA002082E76FF00B003B
:102950007FE7A76917B96FF00C007AE73B699E42E1
:1029600096D03F68F6E7FB7DC8F34012B2EBD31F69
:1029700040F0CE80C3F38403B34240F0CC8006998C
:102980002B7B4FEA981279B3D2073CD4032B40F249
:10299000C580DDE90223C7E902232B7BAE1D033B83
:1029A000DBB23246394604F10C00FFF729FB002860
:1029B00008DA39462046FFF7BFF93846FFF7D0F965
:1029C000032046E7AB883B832A7B033AD2B2B88A1E
:1029D0003146FFF755FAFB7DB882DA43C2F3C012E5
:1029E00062F3C713FB75AFE76AB92E1D013BDBB27B
:1029F0003246394604F10C00FFF702FB0028D8DB11
:102A00002A7B013AE2E7FA8AC2F30902013B052A6E
:102A1000D9B250D8281D002399420AD907EB020EDB
:102A2000013210F801CB8EF81AC00133062ADBB24E
:102A3000F2D1DDE902898B4207F11A02CDE908895A
:102A40000A9238BF04337A680B9234BF5B190023B3
:102A50000C93FB8AADF836A0C3F3090319449DF823
:102A60001C308DF83A309DF814308DF83B3000233F
:102A7000ADF834108DF838B08DF839607B602A7B62
:102A8000B88A013A291DFFF7FBF93B8BB8828342D4
:102A900003D1A36808A92046984708A92046FFF754
:102AA0006DFE3846FFF75CF9B88A3B8B984214BF3D
:102AB00011200020CDE6786810B34FF0060E0368B1
:102AC0009BB9A2EB0E021B2A13D80332024405F174
:102AD000040E1F309942ACD91EF801CB02F801CF89
:102AE00001339042DBB2F5D1A3E70EF11C0E18467C
:102AF000E5E7184B184A194840F2B31101F044FCBD
:102B0000034696E76FF00900A3E66FF00A00A0E61F
:102B10006FF00D009DE66FF00E009AE66FF00F006B
:102B200097E6FB7D68F386036FF3C713FB753946A1
:102B30002046FFF701F9069B002B7FF4D8AEFB7D02
:102B4000C3F38402013262F38603FB7503E700BF1F
:102B500080841E008C4800087046000894490008D4
:102B60002DE9F0414C4EB04240F081804B4CDFF8F3
:102B700030E1E56945F00075E561E469846AD4F8FF
:102B8000007207EA0E0747F00107C4F80072D4F894
:102B9000005205EA0E0545F0010545EA0121C4F899
:102BA0000012002A65D00021C4F81C120F46C4F898
:102BB0000412C4F80C12C4F8141204EBC10501315C
:102BC0000E29C5F84072C5F84472F6D14FF0000ED8
:102BD0004FF0010C964510D1826AD2F80032B04213
:102BE00023F00103C2F8003253D12C4BDA6922F0F2
:102BF0000072DA61DB69BDE8F0819F781D8817F00B
:102C0000010F18BFD4F804820CFA05F11CBF41EA89
:102C10000808C4F8048217F0020F1EBFD4F80C8213
:102C200041EA0808C4F80C827F0742BFD4F8147246
:102C30000F43C4F8147204EBC5055F68C5F8407211
:102C40009F68C5F84472D4F81C522943C4F81C127A
:102C50000C330EF1010EBDE7846A0021C4F81C128A
:102C6000C4F80412C4F80C12C4F81412AEE7002A17
:102C7000F2D1836A0022C3F84022C3F84422C3F889
:102C80000422C3F814220122C3F80C22C3F81C2228
:102C9000A2E7BDE8F08100BF182400200010024028
:102CA0000000FFFF184A916A08B58B688B6013F02B
:102CB000010105D013F00C0F14BF4FF48031012136
:102CC000D80506D513F4406F14BF41F4003141F02C
:102CD0000201D80306D513F4402F14BF41F480211C
:102CE00041F00401D3690BB107489847202383F3CF
:102CF00011880021054800F06DFE002383F3118840
:102D0000BDE8084001F064B8182400202024002009
:102D100038B5124CA36ADD68AA0712D05A6922F0AE
:102D200002025A61A36913B101212046984720236A
:102D300083F3118800210A4800F04CFE002383F33E
:102D40001188EB0606D5A36A1021D960236A0BB15E
:102D500002489847BDE8384001F03AB818240020EE
:102D60002824002038B5124CA36A1D69AA0712D086
:102D70005A6922F010025A61A36913B10221204658
:102D80009847202383F3118800210A4800F022FE8F
:102D9000002383F31188EB0606D5A36A102119617D
:102DA000236A0BB102489847BDE8384001F010B8DB
:102DB000182400202824002038B50F4CA36A5D6831
:102DC0005D602A070AD5032222701A6822F00202E7
:102DD0001A60636A13B10021204698476B0706D535
:102DE000A36A9969236A13B1090403489847BDE8A7
:102DF000384000F0EDBF00BF1824002010B50F4C84
:102E0000204600F091FA0E4BA3620B21132000F034
:102E10006BFA0B21142000F067FA0B21152000F04B
:102E200063FA0B21162000F05FFA002320461A46B1
:102E30000E21BDE81040FFF793BE00BF182400200C
:102E4000006400400F4B984210B5044605D10E4B6C
:102E5000DA6942F00072DA61DB69A36A01221A6062
:102E6000A36A5A68D20707D5626851681268D961A7
:102E70001A60064A5A6110BD0121082000F0DEFCEC
:102E8000EEE700BF18240020001002405B8701001D
:102E900003291AD8DFE801F0020A0F14836A9B683D
:102EA00013F0E05F14BF012000207047836A986828
:102EB000C0F380607047836A9868C0F3C060704751
:102EC000836A9868C0F30070704700207047000064
:102ED00010B503291FD8DFE801F0021F2327816AFC
:102EE0008B68C3F30163183301EB03131078810679
:102EF0001ED55468C0F30011490041EAC40141F0F5
:102F0000040100F00F00586090689860D268DA60A1
:102F100041F00101196010BD836A03F5C073E5E754
:102F2000836A03F5C873E1E7836A03F5D073DDE7CD
:102F30009488C0F30011490041EA4451E1E70000E0
:102F400001290CD003D3022910D000207047836AD6
:102F5000DA68920701D1186903E001207047836A9B
:102F6000D86810F0030018BF01207047836AF2E7A9
:102F700010B539B9836AD96889071BD11B699B07CA
:102F800004D110BD012915D0022948D1816AD1F898
:102F9000C031D1F8C401D1F8C8411461D1F8CC4195
:102FA000546120240C610C69A40717D14C6944F0CA
:102FB000100412E0816AD1F8B031D1F8B401D1F82F
:102FC000B8411461D1F8BC4154612024CC60CC6874
:102FD000A40703D14C6944F002044C6111795C08E8
:102FE00064F304119C0864F34511117189064BBF09
:102FF00091681189DB085B0D4CBF63F31C0163F31F
:103000000A01137948BF916060F3030313714FEA1B
:1030100010234FEA104058BF11811370508010BD2B
:10302000002304491A465A50C8180833802B4260BE
:10303000F9D17047442400200268436811430160BD
:1030400003B1184770470000024A136843F0C003F9
:103050001360704700380140024A136843F0C00310
:1030600013607047004400402DE9F047C66D376893
:10307000F46934620546200719D014F0080F0CBF1C
:1030800000218021E20748BF41F02001A30748BF8B
:1030900041F04001600748BF41F48071202383F371
:1030A0001188281DFFF7C8FF002383F31188E2056C
:1030B0000AD5202383F311884FF40071281DFFF7F0
:1030C000BBFF002383F311884FF020094FF0000A63
:1030D00014F0200831D13B0616D54FF0200905F138
:1030E000380A200610D589F31188504600F0A0FA5E
:1030F00000282FDA0821281DFFF79EFF27F0800304
:103100003360002383F3118879060DD562060BD551
:10311000202383F31188EA6C2B6D9A4201D12B6C2A
:10312000F3B9002383F31188E30621D5AA6E13694E
:10313000F3B15069BDE8F047184789F31188B38CA3
:1031400095F864102846194000F00CFB8AF31188AA
:10315000F469BDE780B2308588F31188F469C0E76F
:103160001021281D27F04007FFF766FF3760D8E7DA
:10317000BDE8F08708B50348FFF776FFBDE80840D3
:1031800000F026BEC424002008B50348FFF76CFFFA
:10319000BDE8084000F01CBE3025002037B51D4CAE
:1031A0001D4D204600F0C4FA009404F114000023E1
:1031B00020221A4900F086F92022009404F13800F8
:1031C000174B184900F000FA174BE3652566174CBA
:1031D0000C21252000F088F8204600F0A9FA04F11F
:1031E0001400009400232022114900F06BF904F12F
:1031F000380000940F4B1049202200F0E5F90F4BE6
:10320000E3650C212620256603B0BDE8304000F0C0
:103210006BB800BFC4240020005125029C2500206B
:1032200049300008DC25002000380140302500200E
:10323000BC25002059300008FC2500200044004037
:10324000254B002908BF1946037C8166012B30B548
:1032500008D1224B984231D1214B9A6942F48042E5
:103260009A619B690A68036EC46D03EB5203B3FB5A
:10327000F2F34A68150442BF23F0070503F0070381
:1032800043EA4503E3608B6843F040036360CB6827
:1032900043F00103A36042F4967343F001032360FB
:1032A00051054FF0FF33236205D512F010220FD0E5
:1032B000B2F1805F0ED080F8643030BD094B984287
:1032C000D0D1074BDA6942F40032DA61DB69C9E731
:1032D0007F23F0E73F23EEE7D0490008C424002015
:1032E000001002403025002000F1604300F01F0272
:1032F000400903F5614309018000C9B200F1604053
:1033000083F8001300F5614001239340C0F8803139
:103310000360704700F16040090100F56D40C9B2DB
:1033200001767047FFF76ABD00F1080201230370C0
:1033300082600023C26000F11002436002614261BA
:103340008361C361036243627047000010B52023AC
:10335000044683F31188022303704160FFF772FD76
:1033600003232370002383F3118810BD2DE9F0415E
:103370001F4604460D461646202383F3118800F1AC
:1033800008082378042B0ED029462046FFF780FD3D
:1033900048B1204632462946FFF79AFD002080F3C7
:1033A0001188BDE8F0813946404600F0F7FA002860
:1033B000E7D0002383F31188BDE8F0812DE9F041C7
:1033C0001F4604460D461646202383F3118800F15C
:1033D00010082378042B0ED029462046FFF7B0FDB5
:1033E00048B1204632462946FFF7C2FD002080F34F
:1033F0001188BDE8F0813946404600F0CFFA002838
:10340000E7D0002383F31188BDE8F081F8B51546B5
:1034100082680669AA420B46816938BF8568761AB8
:10342000B542044607D218462A46FEF745FBA36973
:103430002B44A3610DE011D932461846FEF73CFB40
:10344000AF1B3A46E1683044FEF736FBE2683A4487
:10345000A261A3685B1BA3602846F8BD18462A46F4
:10346000FEF72AFBE368E4E783682DE9F0410446B0
:1034700093421546266938BF85684069361AB542B9
:103480000F4606D22A46FEF717FB63692B44636199
:103490000DE012D93246A5EB0608FEF70DFB4246B9
:1034A000B919E068FEF708FBE26842446261A3686C
:1034B0005B1BA3602846BDE8F0812A46FEF7FCFAB4
:1034C000E368E4E710B50A440024C361029B00608E
:1034D00040608460C160816141610261036210BD2E
:1034E00008B582694369934201D1826882B98268D2
:1034F000013282605A1C42611970426903699A4222
:1035000001D3C3684361002100F058FA002008BDD0
:103510004FF0FF3008BD000070B5202304460E4672
:1035200083F31188A568A5B1A368A269013BA360D4
:10353000531CA36115782269934224BFE368A361F9
:10354000E3690BB120469847002383F3118828468E
:1035500070BD3146204600F021FA0028E2DA85F3FA
:10356000118870BD2DE9F74F05460F4690469A46E3
:10357000D0F81C90202686F311884FF0000B1446DB
:1035800064B1224639462846FFF740FF034668B932
:103590005146284600F002FA0028F1D0002383F3B8
:1035A0001188A8EB040003B0BDE8F08FB9F1000F5B
:1035B00003D001902846C847019B8BF31188E41A79
:1035C0001F4486F31188DBE7C16081614161C361FB
:1035D0001144009B0060406082600161036270479B
:1035E000F8B504460E461746202383F31188A568D4
:1035F000A5B1A368013BA36063695A1C62611E7098
:10360000236962699A4224BFE3686361E3690BB18D
:1036100020469847002080F31188F8BD394620469F
:1036200000F0BCF90028E2DA85F31188F8BD00004B
:10363000836942699A4210B501D182687AB9826879
:10364000013282605A1C82611C7803699A4201D35C
:10365000C3688361002100F0B1F9204610BD4FF02E
:10366000FF3010BD2DE9F74F05460F4690469A46AC
:10367000D0F81C90202686F311884FF0000B1446DA
:1036800064B1224639462846FFF7EEFE034668B984
:103690005146284600F082F90028F1D0002383F338
:1036A0001188A8EB040003B0BDE8F08FB9F1000F5A
:1036B00003D001902846C847019B8BF31188E41A78
:1036C0001F4486F31188DBE70268436811430160F9
:1036D00003B11847704700001430FFF743BF0000E4
:1036E0004FF0FF331430FFF73DBF00003830FFF7D5
:1036F000B9BF00004FF0FF333830FFF7B3BF000011
:103700001430FFF709BF00004FF0FF311430FFF70E
:1037100003BF00003830FFF763BF00004FF0FF32F7
:103720003830FFF75DBF000000207047FFF736BD5F
:10373000044B0360002343608360C3600123037470
:10374000704700BFE849000810B52023044683F302
:103750001188FFF775FD02232374002383F311887A
:1037600010BD000038B5C36904460D461BB90421DD
:103770000844FFF7A9FF294604F11400FFF7B0FE43
:10378000002806DA201D4FF48061BDE83840FFF7BD
:103790009BBF38BD024B00221B605B609A60704784
:1037A0001C260020002303748268054B1B6899685F
:1037B0009142FBD25A6803604260106058607047C3
:1037C0001C26002008B5202383F31188037C032BDB
:1037D00005D0042B0DD02BB983F3118808BD4369A4
:1037E00000221A604FF0FF334361FFF7DBFF002335
:1037F000F2E790E80C001A6002685360F2E70000FC
:10380000002303748268054B1B6899689142FBD8BA
:103810005A68036042601060586070471C260020A0
:10382000054B19690874186802681A6053601861BA
:1038300001230374FCF7E8BE1C26002030B54B1CA6
:1038400087B005460A4C10D023690A4A01A800F047
:10385000DDF82846FFF7E4FF049B13B101A800F050
:10386000EFF82369586907B030BDFFF7D9FFF8E7D3
:103870001C260020C537000838B50C4D41612B6966
:1038800081689A689142044603D8BDE83840FFF742
:1038900089BF1846FFF786FF01232C610146237478
:1038A0002046BDE83840FCF7AFBE00BF1C26002014
:1038B000044B1A681B6990689B68984294BF00206B
:1038C000012070471C26002010B5084C2368206991
:1038D0001A6822605460012223611A74FFF790FF76
:1038E00001462069BDE81040FCF78EBE1C26002072
:1038F00008B5FFF7DDFF18B1BDE80840FFF7E4BFEA
:1039000008BD0000826002220274002242747047E7
:103910008368A3F17C0243F80C2C026943F83C2C29
:10392000426943F8382C074A43F81C2CC26843F814
:10393000102C022203F8082C002203F8072CA3F114
:10394000180070472106000810B5202383F3118862
:10395000FFF7DEFF00210446FFF78EFF002383F30D
:103960001188204610BD0000024B1B6958610F20D2
:10397000FFF756BF1C260020202383F31188FFF792
:10398000F3BF000008B50146202383F31188082007
:10399000FFF754FF002383F3118808BD49B1064B9C
:1039A00042681B6918605A60136043600420FFF787
:1039B00045BF4FF0FF3070471C2600200368984237
:1039C00006D01A680260506059611846FFF7EABED7
:1039D0007047000038B504460D462068844200D187
:1039E00038BD036823605C604561FFF7DBFEF4E7E8
:1039F000054B03F114025A619A614FF0FF32DA610C
:103A000000221A62704700BF1C26002010B5C26059
:103A10000A4A036153699C68A1420CD85C68036040
:103A200044602060586081609868411A99604FF046
:103A3000FF33D36110BD091B1B68ECE71C26002077
:103A4000036881689A680A449A6042681360036850
:103A50005A600023C360024B4FF0FF32DA617047B7
:103A60001C26002000207047FEE700007047000081
:103A70004FF0FF3070470000BFF34F8F024AD3680A
:103A8000DB07FCD4704700BF0020024008B5074B9D
:103A90001B7853B9FFF7F0FF054B1A69120641BFB7
:103AA000044A5A6002F188325A6008BD6C26002030
:103AB000002002402301674508B5054B1B7833B948
:103AC000FFF7DAFF034A136943F08003136108BD6F
:103AD0006C260020002002407F289ABF00F580302D
:103AE000C0020020704700004FF4006070470000E3
:103AF000802070477F2808B50BD8FFF7EDFF00F551
:103B000000630268013204D104308342F9D10120FC
:103B100008BD002008BD00007F2810B504461CD851
:103B2000FFF7AAFFFFF7B2FF0D4BF322DA60022284
:103B30001A61FFF7D1FF58611A6942F040021A6119
:103B4000FFF79AFF4FF4006100F0F6F8FFF7B4FFBB
:103B50002046BDE81040FFF7CDBF002010BD00BFDC
:103B6000002002402DE9F84312F00103144606D06C
:103B7000204B40F243221A600020BDE8F8838518EC
:103B80001D4A954204D91B4A4FF412711160F3E7A4
:103B9000FFF77CFFFFF770FFDFF86C80451A4FF0EE
:103BA0000109012C05EB01060F4604D8FFF784FF3D
:103BB0000120BDE8F883C8F8109031F8023B33804B
:103BC000FFF75AFF0020C8F8100033883A889BB2EC
:103BD0009A420DD0074B40F25F221A60074B1E60DD
:103BE000074B1C60074B1F60FFF766FFBDE8F883BB
:103BF000023CD6E768260020FFFF03085C26002071
:103C0000642600206026002000200240084908B5F4
:103C10000B7828B153B9FFF739FF01230B7008BDAA
:103C200023B1BDE808400870FFF746BF08BD00BFDC
:103C30006C26002038B500F079F90D4B0D4A1C6A4E
:103C400011684FF47A7303FB04F38B420A49D1E9FC
:103C5000004504D2003445F10105C1E90045E418EE
:103C600045F10005136000F06BF92046294638BD88
:103C70001C260020702600207826002008B5FFF7BB
:103C8000D9FF4FF47A720023FCF7A2FA08BD00BFF7
:103C900010B50244064B0439D2B2904200D110BD97
:103CA000441C00B253F8200041F8040FE0B2F4E7DE
:103CB00050280040104B30B51C6A240407D41C6AFD
:103CC00044F440741C621C6A44F400441C620B4CB3
:103CD000236843F4807323600244094B0439D2B251
:103CE000904200D130BD441C00B251F8045F43F84B
:103CF0002050E0B2F4E700BF001002400070004026
:103D00005028004007B5012201A90020FFF7C0FF9D
:103D1000019803B05DF804FB13B50446FFF7F2FF0A
:103D2000A04206D002A9012241F8044D0020FFF76D
:103D3000C1FF02B010BD000070470000074B45F204
:103D400055521A6002225A6040F6FF729A604CF691
:103D5000CC421A60024B01221A70704700300040BA
:103D600081260020034B1B781BB1034B4AF6AA2285
:103D70001A6070478126002000300040034B1B680A
:103D80009B0042BF024B01221A7070472410024070
:103D900080260020024B4FF080721A60704700BFEF
:103DA00024100240014B1878704700BF8026002085
:103DB000064A536823F001035360EFF30983683325
:103DC00083F30988002383F31188704730EF00E004
:103DD00010B5202383F31188104B5B6813F4006344
:103DE00018D0F1EE103AEFF309844FF0807344F8E5
:103DF0004C3C0B4BDB6844F8083CA4F1680383F3AC
:103E00000988FFF755FD18B1064B44F8503C10BD2A
:103E1000054BFAE783F3118810BD00BF00ED00E009
:103E200030EF00E03106000834060008704700005B
:103E3000FEE70000084A094B09498B4204D3094AAE
:103E40000021934205D3704752F8040F43F8040B46
:103E5000F3E743F8041BF4E79C4B0008C427002059
:103E6000C4270020C4270020FEE7000010B5174C2F
:103E7000FFF790FCFFF7BCFD802215492046FFF7B5
:103E800041FD012344F8180C0374124B124AD968FF
:103E900021F4E0610904090C0A431049DA60CA6898
:103EA00042F08072CA600E490A6842F001020A605C
:103EB0001022DA77202283F82220002383F311884E
:103EC00062B60848BDE81040FFF73EBD442600201A
:103ED000104A000800ED00E00003FA05F0ED00E0F4
:103EE000001000E0184A0008F8B50F4C226A0132B1
:103EF0002262224652F8141F9142154606D08B6862
:103F0000013B8B60202663699A6802B1F8BD19688D
:103F1000DF68DA604D60616182F311881869B84723
:103F200086F31188EFE700BF1C260020EFF3118015
:103F300020B9EFF30583202282F311887047000037
:103F400010B558B9EFF30584C4F3080414B180F335
:103F5000118810BDFFF7CCFC84F3118810BD000060
:103F60004B6843608B688360CB68C3600B694361B7
:103F70004B6903628B6943620B6803607047000002
:103F800008B5194B9A6A42F4FC029A629A6A22F4C2
:103F9000FC029A629A6A5A6942F4FC025A61134A14
:103FA0005B6911464FF09040FFF7DAFF104802F1CD
:103FB0001C01FFF7D5FF0F4802F13801FFF7D0FFD2
:103FC0000D4802F15401FFF7CBFF0C4802F17001DC
:103FD000FFF7C6FF0A4802F18C01FFF7C1FFBDE8F9
:103FE000084000F065B800BF00100240384A0008E1
:103FF0000004004800080048000C00480010004879
:104000000014004808B500F08FF9FFF72FFFBDE856
:104010000840FFF7B3BE00007047000010B5214C08
:10402000A26A62F4FC02A262A26A02F4FC02A26228
:104030004FF0FF31A26A22692161226900222261C8
:104040002069E068E160E168E260E168E1691648E2
:1040500041F08051E161E169016841F480710160E2
:10406000216A01F44071B1F5407F1EBF4FF48033E7
:1040700023622262236A1B0407D4236A43F4407339
:104080002362236A43F40043236200F02DF9A369FD
:10409000064A43F00103A361A369136843F02003B8
:1040A000136010BD0010024000700040000001408D
:1040B0001C4B1A6842F001021A601A689007FCD57E
:1040C0005A6822F003025A605A6812F00C02FBD1BF
:1040D000196801F0F90119605A601A6842F48032D7
:1040E0001A601A689103FCD50F4A5A604FF40452C3
:1040F000DA6230221A631A6842F080721A601A6813
:104100009201FCD5094A122111605A6842F002025C
:104110005A605A6802F00C02082AFAD11A6B1A6324
:10412000704700BF0010024000241D000020024024
:10413000084A08B5536911680B4003F00103536145
:1041400023B1054A13680BB150689847BDE8084091
:10415000FFF73EBE0004014044240020084A08B591
:10416000536911680B4003F00203536123B1054A00
:1041700093680BB1D0689847BDE80840FFF728BEA8
:104180000004014044240020084A08B5536911681E
:104190000B4003F00403536123B1054A13690BB1CB
:1041A00050699847BDE80840FFF712BE000401407F
:1041B00044240020084A08B5536911680B4003F0F5
:1041C0000803536123B1054A93690BB1D06998473D
:1041D000BDE80840FFF7FCBD000401404424002076
:1041E000084A08B5536911680B4003F01003536186
:1041F00023B1054A136A0BB1506A9847BDE80840DD
:10420000FFF7E6BD0004014044240020174B10B521
:104210005C691A68144004F478725A61A30604D5E4
:10422000134A936A0BB1D06A9847600604D5104AC6
:10423000136B0BB1506B9847210604D50C4A936B56
:104240000BB1D06B9847E20504D5094A136C0BB14A
:10425000506C9847A30504D5054A936C0BB1D06CFC
:104260009847BDE81040FFF7B3BD00BF0004014010
:10427000442400201A4B10B55C691A68144004F4F9
:104280007C425A61620504D5164A136D0BB1506D1C
:104290009847230504D5134A936D0BB1D06D984709
:1042A000E00404D50F4A136E0BB1506E9847A10479
:1042B00004D50C4A936E0BB1D06E9847620404D5B6
:1042C000084A136F0BB1506F9847230404D5054A71
:1042D000936F0BB1D06F9847BDE81040FFF778BDE2
:1042E0000004014044240020062108B50846FEF7DA
:1042F000FBFF06210720FEF7F7FF06210820FEF747
:10430000F3FF06210920FEF7EFFF06210A20FEF742
:10431000EBFF06211720FEF7E7FF06212820BDE866
:104320000840FEF7E1BF000008B5FFF777FEFEF793
:1043300077FEFEF7F7FFFFF7F9F9FFF76DFEBDE82F
:10434000084000F001B8000000F00EB808B52023C6
:1043500083F31188FFF7C8FD002383F31188BDE8BC
:104360000840FFF735BD0000054B064A5A600022A1
:104370009A6007221A6008210B20FEF7CBBF00BF0E
:1043800010E000E03F1901001FB51C46094B1B68F7
:104390000546D86852B1084B02928DE80A002246C1
:1043A0002B460649FDF7C2FB00F042F8044B1A46C3
:1043B000F2E700BF14110020E04A0008ED4A0008AF
:1043C0004B45000810B501390244904201D100204C
:1043D00010BD10F8013B11F8014FA342F5D0181B96
:1043E00010BD00002DE9F8430746884691461E4659
:1043F0008BB10D46A8EB0500B54207EB000402D2D5
:104400000020BDE8F883324649462046FFF7DAFF30
:1044100018B1013DEEE7BDE8F8832046BDE8F8831A
:10442000034611F8012B03F8012B002AF9D170473C
:1044300008B5062000F02CF80120FFF715FB00005E
:104440001F2938B504460D4604D9162303604FF0E2
:10445000FF3038BD426C12B152F821304BB92046C2
:1044600000F030F82A4601462046BDE8384000F00A
:1044700017B8012B0AD0591C03D116230360012061
:1044800038BD002442F8254028469847002038BD12
:10449000024B01461868FFF7D3BF00BF141100207C
:1044A00038B5074C00230546084611462360FFF740
:1044B000DFFA431C02D1236803B12B6038BD00BF73
:1044C000C0270020FFF7CEBA1210121312110000FD
:1044D00040A2E4F1646891064E6F20617070207311
:1044E00069670A00426164206677206C656E6774B4
:1044F000682025750A0042616420626F6172645F02
:1045000069642025752073686F756C64206265206E
:1045100025750A0042616420617070204352432077
:104520003078253038783A3078253038782030782F
:10453000253038783A3078253038780A00476F6F60
:1045400064206669726D776172650A0072656365E1
:10455000697665645F756E697175655F69645F6CC6
:10456000656E203C2055415643414E5F50524F549A
:104570004F434F4C5F44594E414D49435F4E4F446A
:10458000455F49445F414C4C4F434154494F4E5F56
:10459000554E495155455F49445F4D41585F4C4523
:1045A0004E475448002E2E2F2E2E2F546F6F6C73B3
:1045B0002F41505F426F6F746C6F616465722F633F
:1045C000616E2E63707000616C6C6F636174656402
:1045D0005F6E6F64655F6964203C3D203132370057
:1045E0006F72672E6172647570696C6F742E6633BA
:1045F00030335F4D6174656B47505300766F69646B
:104600002068616E646C655F616C6C6F6361746976
:104610006F6E5F726573706F6E73652843616E6154
:104620007264496E7374616E63652A2C2043616EF7
:1046300061726452785472616E736665722A2900E1
:1046400053544D33324633787800000063616E6115
:104650007264496E6974000063616E6172645365CF
:10466000744C6F63616C4E6F6465494400000000D8
:1046700063616E61726448616E646C655278467203
:10468000616D650063616E6172644465636F64654A
:104690005363616C6172000063616E617264456EA8
:1046A000636F64655363616C61720000696E63726D
:1046B000656D656E745472616E736665724944000F
:1046C000656E717565756554784672616D657300C8
:1046D0007075736854785175657565007072657092
:1046E000617265466F724E6578745472616E73665E
:1046F00065720000636F707942697441727261790A
:1047000000000000646573636174746572547261C3
:104710006E736665725061796C6F616400000000B1
:1047200066726565426C6F636B0000006269745F5E
:104730006C656E677468203E20300072656D61693B
:104740006E696E675F62697473203E203000696E27
:104750007075745F6269745F6F6666736574203E1E
:104760003D20626C6F636B5F6269745F6F66667336
:10477000657400626C6F636B5F656E645F62697421
:104780005F6F6666736574203E20626C6F636B5F5B
:104790006269745F6F66667365740072656D6169E6
:1047A0006E696E675F6269745F6C656E67746820BE
:1047B0003C3D2072656D61696E696E675F62697408
:1047C0007300696E7075745F6269745F6F6666739B
:1047D0006574203C3D207472616E736665722D3E77
:1047E0007061796C6F61645F6C656E202A2038009F
:1047F0006F75747075745F6269745F6F66667365F8
:1048000074203C3D2036340072656D61696E696EBE
:10481000675F6269745F6C656E677468203D3D20F8
:10482000300028726573756C74203E203029202674
:10483000262028726573756C74203C3D203634291F
:104840002026262028726573756C74203C3D2062FA
:1048500069745F6C656E67746829000064657374C1
:10486000696E6174696F6E20213D202828766F691A
:1048700064202A2930290076616C756520213D204D
:104880002828766F6964202A293029006F666673AC
:1048900065745F77697468696E5F626C6F636B20C3
:1048A0003C2028333255202D205F5F6275696C747F
:1048B000696E5F6F66667365746F66202843616E0C
:1048C000617264427566666572426C6F636B2C2020
:1048D00064617461292900006F75745F696E7320CB
:1048E000213D202828766F6964202A29302900007C
:1048F0007372635F6C656E203E20305500000000CF
:104900002863616E5F696420262030783146464610
:10491000464646465529203D3D2063616E5F6964E9
:1049200000000000616C6C6F6361746F722D3E73E8
:104930007461746973746963732E63757272656EE2
:10494000745F75736167655F626C6F636B73203E44
:10495000203000007472616E736665725F69642056
:10496000213D202828766F6964202A2930290000FB
:1049700073746174652D3E6275666665725F626C04
:104980006F636B73203D3D202828766F6964202A71
:10499000293029002E2E2F2E2E2F6D6F64756C65F9
:1049A000732F6C696263616E6172642F63616E6103
:1049B00072642E63006974656D2D3E6672616D656B
:1049C0002E646174615F6C656E203E2030000000D3
:1049D0000096000000000000000000000000000041
:1049E000000000000000000000000000F536000894
:1049F000E13600081D3700080937000815370008A0
:104A000001370008ED360008D936000829370008BC
:104A10006D61696E00000000304A000888260020A1
:104A2000C027002001000000693E000800000000CF
:104A300069646C6500000000A001A802000000008D
:104A4000FAAABEAA50001400EFFF00000077000091
:104A5000709709000000A00000000000AAAAFAAAAE
:104A600000005000FFFF0000000000000077000081
:104A70000000000000000000AAAAAAAA000000008E
:104A8000FFFF000000000000000000000000000028
:104A900000000000AAAAAAAA00000000FFFF000070
:104AA0000000000000000000000000000000000006
:104AB000AAAAAAAA00000000FFFF00000000000050
:104AC000000000000000000000000000AAAAAAAA3E
:104AD00000000000FFFF00000000000000000000D8
:104AE0002C2066756E6374696F6E3A200061737373
:104AF000657274696F6E2022257322206661696C6D
:104B000065643A2066696C6520222573222C206C2E
:104B1000696E65202564257325730A00E4B6FF7F5E
:104B20000100000000000000FFFFFFFF6400000024
:104B300000000000FE2A0100D2040000181100202D
:104B40000000000000000000000000000000000065
:104B50000000000000000000000000000000000055
:104B60000000000000000000000000000000000045
:104B70000000000000000000000000000000000035
:104B80000000000000000000000000000000000025
:104B90000000000000000000000000000000000015
:00000001FF
